:1000000090C00020950600009306000093060000B3
:100010009306000093060000930600000000000015
:100020000000000000000000000000009306000037
:1000300093060000000000009306000093060000F5
:10004000930600009306000093060000930600004C
:10005000930600009306000093060000930600003C
:10006000930600009306000093060000D5070000E9
:10007000930600009306000093060000930600001C
:10008000930600009306000093060000930600000C
:1000900093060000930600009306000093060000FC
:1000A00093060000930600009306000093060000EC
:1000B00093060000930600009306000093060000DC
:1000C00093060000930600009306000093060000CC
:1000D00093060000930600009306000093060000BC
:1000E00093060000930600000000000000000000DE
:1000F000000000005906000093060000930600006F
:10010000930600009306000093060000930600008B
:10011000930600009306000093060000930600007B
:10012000930600009306000093060000930600006B
:10013000930600009306000093060000930600005B
:10014000930600009306000093060000930600004B
:10015000930600009306000093060000930600003B
:10016000930600009306000093060000930600002B
:10017000930600009306000093060000930600001B
:10018000930600009306000093060000930600000B
:1001900093060000930600009306000093060000FB
:1001A00093060000930600009306000093060000EB
:1001B00093060000930600009306000093060000DB
:1001C00093060000930600009306000093060000CB
:1001D00093060000930600009306000093060000BB
:1001E00093060000930600009306000093060000AB
:1001F000930600009306000093060000930600009B
:10020000930600009306000093060000930600008A
:10021000930600009306000093060000930600007A
:10022000930600009306000093060000930600006A
:10023000930600009306000093060000930600005A
:10024000930600009306000093060000930600004A
:10025000930600009306000093060000930600003A
:100260009306000010B5054C237833B9044B13B145
:100270000448AFF300800123237010BD000000206C
:1002800000000000040F000008B5034B1BB1034938
:100290000348AFF3008008BD000000000400002008
:1002A000040F000038B5044600380C4B0D4618BF4B
:1002B00001200B494FF4E07298472368AB4208D005
:1002C0004BB9084B25602046984740F2B273A361B2
:1002D00038BD0020FCE76FF01100F9E75904000079
:1002E000140E00005907000038B50D46044610B141
:1002F000081E18BF01200A490A4B41229847204690
:10030000094B40F8045F29469847002807DB4FF463
:100310000043A382054B2361054BE360002038BDF9
:100320002E0E000059040000950B0000A9030000E8
:100330007103000030B50C4685B0054610B1081EAB
:1003400018BF0120B4220749074B9847236801933F
:1003500063680293A368039301A9044B281D98477F
:1003600005B030BD2E0E000059040000C90C00007D
:100370007FB50446003818BF01200E4615460749D0
:10038000074BA42298470023CDE9016301A9054B3F
:100390000395A4F10C00984704B070BD2E0E000028
:1003A00059040000350300007FB50446003818BF2B
:1003B00001200E4615460749074B8822984700231F
:1003C000019301A9054B0296A4F10C0003959847EF
:1003D00004B070BD2E0E000059040000350300006B
:1003E000094A138810B59BB21380084B9847084BF5
:1003F0009847084B9847084B9847BDE81040074B73
:1004000040F6FF70184700BF004000413107000070
:10041000610400004D060000790400002104000082
:10042000C20707D5094B0A4A1A6243F6FD7259689A
:100430001142FCD1030707D5044B064ADA6243F6A2
:10044000FD7259681142FCD1704700BF001C00408A
:10045000010101000501010000B900BE7047000064
:10046000034B044A9A611A699207FCD5704700BF92
:1004700000100040062600032C4A136A23F00F03E5
:1004800043F00403136243F6FD7351681942FCD133
:1004900053685807C3F38001FAD4254B254A1977CE
:1004A0009A6293F82C20C2F30011D206F9D483F893
:1004B00020101F4B93F82C205007FBD402221A77F0
:1004C0001B4B93F82C209107FBD45A6A5A62184BA5
:1004D00093F82C201207FBD49F2283F82020144B82
:1004E00093F82C205007FBD493F82020D10719D57E
:1004F0001A6902F41062B2F5106FF9D10B4A536811
:10050000002BFCD1136A23F00F0343F001031362A5
:1005100043F6FD7351681942FCD1044A53685B07E6
:10052000FCD470471A69D205FCD5E7E7001C0040EF
:1005300000100040000001042DE9F8430E46154666
:10054000044618B129B3101E18BF01201249134BDD
:10055000134FF12298470834B9462046B84700287F
:10056000FBD0DFF844800027F15D2046C0472046DD
:10057000C8470028FBD00137BD42F5D8002D094EF1
:1005800008BF01252046B0470028FBD02846BDE81B
:10059000F8830846DAE700BF4A0E0000590400005D
:1005A000770B0000810B0000690B00002DE9F84378
:1005B0000E461546044618B1E9B1101E18BF0120B9
:1005C0000E490F4BDFF83C90DFF83C804FF4867209
:1005D0009847002708342046C8470028FBD020460B
:1005E000C047F0550137BD42F5D8002D14BF28464D
:1005F0000120BDE8F8830846E2E700BF4A0E00008C
:10060000590400008B0B00006F0B000038B50D463D
:10061000044610B1081E18BF01200749074B3422B9
:100620009847074B294604F10800984718B9054B2D
:100630006360054B236038BD4A0E0000590400007A
:100640003D0B0000AD05000039050000014B012203
:100650005A717047000800400B4A937882B0DBB2B1
:100660000193019B990705D5084B1B6813B150688E
:1006700002B01847019BDB0704D5044B5B680BB144
:10068000014AF4E702B07047000002411C0000205C
:100690007047FEE718491948814210B50AD0184B37
:1006A000DA1C121A22F00302C41EA34238BF002231
:1006B000144B9847144B1548DA1C121AC11E22F02D
:1006C0000302994288BF0022114B00219847114A2A
:1006D000114B22F07F029A60D3F8882042F4700216
:1006E000C3F88820BFF34F8FBFF36F8F0B4B984732
:1006F0000B4B9847FEE700BF040F000000000020EE
:1007000000000020E90D0000900000200000002003
:10071000050E00000000000000ED00E0A10D00004B
:100720002507000008B5014B9847FEE7890D00003A
:10073000064B42F286029A8200229A75DA75DA69CD
:1007400002F47C52DA6101221A74704700140040EE
:1007500003690B42FCD1704710B5044618B100681C
:10076000003818BF01201749174B2F229847174B05
:100770002068174A1C6048F20301904703889B07D2
:100780000AD52068038823F002031B041B0C038096
:100790009047206802219047206803889BB243F06D
:1007A00001030380012190472068904720684FF49F
:1007B0000143038048F20301904723680020186634
:1007C00010BD00BF660E0000590400002C00002080
:1007D000510700000D4B10B51C68226891895389A0
:1007E0009BB20B40DA0507D563682046984723681B
:1007F0004FF480729A8110BD5B04FCD5A36820463B
:10080000984723684FF48042F4E700BF2C00002093
:1008100000F01F0330B501259D4040090D4BC0017C
:100820000229ACB24FEA154203440BD044F0804495
:1008300044F4003442F040425D6042F400329C6275
:100840009A6230BD44F080449D6042F040429C6218
:10085000F6E700BF00800041420900F01F0303EBF0
:10086000C21303F1824303F5004393F8402002F0E2
:10087000FB0283F8402070474309DB0103F1824308
:1008800030B503F5004300F01F041D1903EB5403BA
:1008900095F8402002F0FE0242F0010285F8402067
:1008A000CAB293F8301010F0010F1BBF01F00F0116
:1008B00041EA021101F0F001C9B208BF114383F807
:1008C000301030BD024A536943F4007353617047DE
:1008D0000008004010B5044B044905489847BDE89E
:1008E0001040044B184700BFC5080000002400401A
:1008F00030000020A502000010B5054C0549042079
:10090000A04723460449BDE810400520184700BF12
:10091000790800000300040003000500064B402294
:10092000C3F89C204322C3F88C20044A536943F443
:1009300080535361704700BF001C00400008004016
:1009400010B5054B054906489847064B00229847C5
:10095000BDE81040044B18471D090000003000405E
:10096000500000200D060000F908000070B5124E7E
:10097000124D134C4FF48033C6F81431022150202D
:10098000A84701F5A0015020A0474FF40033C6F856
:10099000143102215120A84701F5A2015120A0479E
:1009A00001215220A847074B074952209847234668
:1009B000BDE87040184700BF0080004111080000EA
:1009C000790800005908000002005200064B40223E
:1009D000C3F810214322C3F88C20044A136A43F061
:1009E00004031362704700BF001C00400008004071
:1009F00010B5054B054906489847064B9847BDE892
:100A00001040054B184700BFCD0900000008004307
:100A10005C000020E90200006D09000010B5054BE4
:100A20009847054B9847054B9847BDE81040044B45
:100A3000184700BFE1030000D5080000410900008D
:100A4000F1090000C3690B42FCD17047C3690B4236
:100A5000FCD170470268034B22F0020202600321BE
:100A6000184700BF450A00000268034B22F002024B
:100A700002600321184700BF4D0A000070B50C4DFD
:100A800006460FCD88B06C460FC495E80F0084E889
:100A90000F006A46002352F8041BB14202D1D8B2BB
:100AA00008B070BD0133082BF5D10020F8E700BF76
:100AB000980E000038B51A4B0446984728B11949DA
:100AC000194B40F2472200209847E369174D13F075
:100AD000010F0ED103212046A84723689B0703D5A9
:100AE000134B98470221A847052323600321204682
:100AF000A84720460121A8470E4B23600321A847A1
:100B00004FF4403363601F21A8470B4BA3604FF69F
:100B1000B943A3810023A373184684F8303038BD4D
:100B20007D0A00007B0E0000590400004D0A000001
:100B3000690A0000040010400200700070B505460C
:100B400000380C46054B064918BF0120BB229847C8
:100B50002C602046034BBDE8704018475904000044
:100B60007B0E0000B50A00000368996270470368B5
:100B7000986AC0B270470368187E00F001007047A1
:100B80000368187EC0F3400070470368187EC0F306
:100B9000800070472DE9F843444B454D0746084611
:100BA0000C469847062818BF0025002F5DD0201E50
:100BB00018BF01203F4E404940F63F12B047B046B3
:100BC000002D70D0E3693D4E13F0010F13D10321C6
:100BD0002046D5F80090B04723689B0709F01C0910
:100BE00003D5374B98470221B04749F001032360F2
:100BF00003212046B04701212046B0472B68DFF88B
:100C0000C4903C6003F01C03082B30D12A4901201A
:100C100040F61D12C0472B6803EA09032360032135
:100C20002046B0476B6823F4083323F4107343F471
:100C3000003343F4107363601721B047AB686362FD
:100C40006B7B84F83030E369002BFCD16B6813F0C8
:100C5000070F0CBF012302233B71AB7BEA7B43EA06
:100C60000223FB800020BDE8F8833846A2E7124942
:100C7000012040F60912C0472B6803EA09032360EC
:100C800003212046B0476B6823F4383323F41073F4
:100C900043F4003363601721B0472B7B23736B7BD6
:100CA00084F83030D2E76FF00C00DCE77D0A0000FA
:100CB000D00E0000590400007B0E0000450A000021
:100CC000550A0000FCFEFFFF2DE9F843046890F888
:100CD00004802A4B0746201ED1E9006540F6A32276
:100CE00018BF0120894626499847E26912F0070299
:100CF0003ED1244B032120469847236899073AD5D3
:100D00001146237ED8B25B070FD48A4218D8C30796
:100D100016D5FB8836B1B8F1010F33788CBF36F8A1
:100D2000023B01360132A3620AE0A36A3DB1B8F189
:100D3000010F2B7085BF1B0A6B7001350235013125
:100D4000000607D4D9F808309342DAD88B42D8D8B5
:100D5000104606E04FF6FF736383802323766FF01F
:100D60001200237E9B07FCD003232376BDE8F88383
:100D70006FF00300FAE76FF01300F7E75904000083
:100D80007B0E0000450A000010B5034B9847BDE8F4
:100D90001040024B184700BF1D0A000091060000DA
:100DA00070B50D4D0D4C641BA4100026A64209D150
:100DB0000B4D0C4C00F096F8641BA4100026A642C4
:100DC00005D170BD55F8043B98470136EEE755F85C
:100DD000043B98470136F2E7F00E0000F00E0000E9
:100DE000F00E0000F40E00000A44914200F1FF33BF
:100DF00000D1704710B511F8014B03F8014F914233
:100E0000F9D110BD02440346934200D1704703F864
:100E1000011BF9E72E2E2F68616C2F7372632F6808
:100E2000616C5F63616C656E6461722E63002E2E6F
:100E30002F68616C2F7372632F68616C5F737069C8
:100E40005F6D5F73796E632E63002E2E2F68616C69
:100E50002F7372632F68616C5F75736172745F7357
:100E6000796E632E63002E2E2F68706C2F72746360
:100E70002F68706C5F7274632E63002E2E2F687063
:100E80006C2F736572636F6D2F68706C5F73657222
:100E9000636F6D2E6300000000300040003400409E
:100EA00000200141004001410000004300040043D4
:100EB00000080043000C0043000000000000000098
:100EC0000000000000000000000000000000000022
:100ED0000C0020000000020000000000FE00FF01E6
:100EE00006000000F8B500BFF8BC08BC9E4670477D
:100EF00089020000F8B500BFF8BC08BC9E467047E8
:040F00006502000086
:00000001FF
